:030000000200807B
:10008000C2AF75814F7590FF75B0FF7520007EFF80
:100090009193C294C2957E5291937B03D295E59041
:1000A00054F04403F590C2957E029193DBEED29515
:1000B000E59054F04402F590C2957E029193782821
:1000C000919C780C919C7806919C91DCD29630960C
:1000D000030206B19006F71204E578C0919C9007E0
:1000E000041204E57B0A510CDBFC91DC90071291B1
:1000F000E57BA1D119852F2B852E2A7BA2D11985CD
:100100002F29852E287BACB1E2E52F54FEF527FB85
:10011000B1807BEEB16379507EFF9193D9FA7BAACF
:10012000D11978C0919C9007221204E5510C510C12
:10013000510C510C7BEEB163D297D29630960302EC
:1001400006B191DC90078491E530B7FD510C78C081
:10015000919C9007631204E520B50302022420B7A6
:10016000F730B7FD510C78C0919C9007431204E51D
:1001700030B50620B7FA0201A9852B26852A257BF2
:10018000ACB1E2E52F544024FF9202510C9007439A
:1001900071B585262B85252A7BA1B1AB300307E5F8
:1001A00027549EFBB18002013430B7FD510C78C05A
:1001B000919C9007531204E530B50620B7FA02016E
:1001C000F18529268528257BACB1E2E52F54202432
:1001D000FF9202510C90075371B585262985252879
:1001E0007BA2B1AB300307E527549EFBB18002012F
:1001F0003430B7FD510C78C0919C9007731204E520
:1002000030B50620B7FA02014902036C7F027EFF77
:100210007DFF02021B7F017E7F7DFFDDFEDEFCDFB6
:10022000FA2280FE7524C975230075227D75210090
:1002300091DC90079391E5788D919C78DF91BD7862
:10024000C0919C9007A391E5510CD2963096030281
:1002500006B17BACB1E2E52F548020B50302036701
:1002600070E8A2B2B392977BAAD119852F2D852E63
:100270002C7887919CD156E52D335008E5243340E6
:10028000110202B6E524335009852D24852C230262
:1002900002B0E52DB52408E52CB523030202B650C3
:1002A000030202B6852D24852C2385242F85232E39
:1002B00078C7919CD156E52D334008E52233501183
:1002C0000202F5E522334009852D22852C21020208
:1002D000E3E522B52D08E521B52C030202F5500314
:1002E0000202F5852D22852C2185222F85212E784D
:1002F000C0919CD156E52B335008E52D33400B02BD
:10030000031CE52D335003020328E52DB52B08E52A
:100310002CB52A0302031C500302032890074378DC
:10032000CD919C91E502024AE529335008E52D3331
:10033000400B02035BE52D33500302034FE529B563
:100340002D08E528B52C0302034F500302035B90F0
:10035000075378CD919C91E502024A9007C578CE6B
:10036000919C91E502024A510C02013491DC900704
:10037000731204E578C0919C9007B41204E5510C07
:1003800078CC919CE52754026007783191BD020337
:1003900095783091BD30B30930B40630B50E020304
:1003A00095E5276402F527510C020380AB27B18045
:1003B000510C02013491DC91E578C0919C90079337
:1003C00091E578CD919C78DF91BD30020A788F91CC
:1003D0009C782191BDC20278C7919C85262F8525E6
:1003E0002ED156511530B40A30B35C30B503020338
:1003F000E522E52664C97007E52570030203E5D20E
:1004000003C297788F919C782091BDE5268525F0D1
:1004100025F06018E5265480701BE52560067525DB
:10042000000203D715267525800203D77526FF75B0
:1004300025800203D7E52560067525000203D775E0
:10044000258015260203D7E526647D7007E5257013
:10045000030203E5D203C297788F919C782091BD67
:10046000E5265480701BE5256008752500052602E9
:1004700003D77525800203D77526FF7525800203F3
:10048000D7E525600875250005260203D775258068
:100490000203D77F18DFFE0000DEF822C294D29557
:1004A000E59054F0F9E8C4540F49F590C295D295FF
:1004B000E8540F49F590C2957E02919322D294D2CE
:1004C00095E59054F0F9E8C4540F49F590C295E8C9
:1004D000540F49F590C2957E029193227801919C28
:1004E0007E22919322E493F891BDA3E49370F822C5
:1004F000D2B10000D2B00000C2B10000C2B022D21E
:10050000B00000D2B1227908C3E8334005C2B1027D
:100510000514D2B100D2B00000C2B0D9EDD2B122E0
:10052000C2007914D2B030B104D9FBD200C2B022DB
:100530007908C3E4D2B00000A2B1C2B0000033D940
:10054000F3F8D2B122C2B10000D2B00000C2B000B4
:1005500000D2B122D2B10000D2B00000C2B000007F
:10056000D2B12291F07890B106B12030000302069A
:10057000D0EBF8B106B1203000030206D091FF2283
:10058000C20391F07890B106B1203000030206D08A
:1005900078ACB106B1203000030206D0EBF8B1060A
:1005A000B1203000030206D091FF2291F07890B183
:1005B00006B1203000030206D0EBF8B106B12030BE
:1005C00000030206D0E526F8B106B1203000030290
:1005D00006D0E525F8B106B1203000030206D0911F
:1005E000FF22752F00752E0091F07890B106B12092
:1005F0003000030206D0EBF8B106B1203000030250
:1006000006D091F07891B106B1203000030206D0F7
:10061000B130882FB15491FF22752F00752E0091B3
:10062000F07890B106B1203000030206D0EBF8B1AB
:1006300006B1203000030206D091F07891B106B1E6
:10064000203000030206D0B130882FB145B1308888
:100650002EB15491FF22E52F54806011E52FC394F1
:1006600001F4F52FD201782D91BD020673C20178F5
:100670002B91BDAB2FEB75F064842430F8ABF09177
:10068000BDEB75F00A842430F8ABF091BD30010861
:10069000E52E6004EB60011BEB2430F891BD782E51
:1006A00091BDE52E23540175F005A42430F891BDC9
:1006B0002291DC9007C891E578C0919C9007D99170
:1006C000E5C29779287EFF9193D9FAB2970206C3C3
:1006D00091DC9007321204E578C0919C9007EA12F1
:1006E00004E5C29779287EFF9193D9FAB29720B595
:0706F000030200800206E492
:0D06F70020202020445331363231202D00C8
:0E07040020202050726F6772616D6D6572006B
:1007120020436869702054657374696E67202100F4
:100722002043686970203C3C204F4B203E3E200015
:100732002043686970203C3C4552524F523E3E2055
:0107420000B6
:10074300205448202D205265676973746572200018
:1007530020544C202D205265676973746572200004
:100763002020546865726D6F6D657465722020007A
:100773004F757470757420506F6C61726974792051
:010783000075
:0F078400202D204D2045204E20552045202D00B2
:100793002054656D70203A2B3030302E30B043003A
:1007A3002D3030302E30202B3030302E30202D2D78
:0107B3000045
:1007B4002020204F7574707574203D202020202047
:0107C4000034
:0307C5002D2D00D7
:1007C800202D204C6F7720426174742E202D20201C
:0107D8000020
:1007D900696E73657274206E657720626174742E18
:0107E900000F
:1007EA00202070757368202D454E5445522D2120C6
:0107FA0000FE
:00000001FF
